:103630009002A1E0FF900296E06F227B017A02796E
:1036400037900120740DF02290021A12120D898217
:033650008A832248
:06369800AE071FEE601AF0
:10369E009000F37444F0A3745CF09000F374FFF5A3
:0A36AE00F01211DB45F060E280F03D
:0136B80022EF
:1036B900E4FFE4FCFD0DBD00010CBC13F8BD88F569
:1036C900E5C130E504E4FF80010FEFD394FA40E24D
:0136D90022CE
:10129B00E4F5D975FF8075EF029002A17421F0126D
:1012AB0037E01233F4E490029EF0D2AF43E601FF35
:1012BB00E490029FF0A3F0C2AF90029EE06009E4BD
:1012CB00A3F0A3F090029EF0D2AF90029FE475F0D2
:1012DB00011211C5C39002A0E094FF90029FE0940D
:1012EB00FF40D40FEFB402C8C2AF53E6FE12373D36
:1012FB0012398212153C1232801235E5D2AF43E619
:10130B00011236B9E49000F1F09000F1E0FFC394C4
:10131B0004500512153280F1123AA3EF6010123609
:10132B0076122D313009F1C2091206A780EA122973
:10133B00CD90027DE07002A3E0603090027D74FFDF
:10134B00F5F01211C590027DE07002A3E0700A90D7
:10135B0002A1E0FF7D13123B3F30170FE490027D9B
:10136B00F0A3F0A214B39214123280123570EF7006
:10137B000302140712311AEF12124213A20113A720
:10138B000213AC0413C10813EC0913F30A13D610A0
:10139B0013DE20000013FB1239FA80541238E6805A
:1013AB004F900237E07005740DF0802212363B7DB2
:1013BB00FF1234228018900237E0B40D04E4F08061
:1013CB000812363B7D011234228003123BBF1232CE
:1013DB0080801D90027D7488F0A374B8F0C21780D2
:1013EB000F1236487F0180051236487FFF12126CB0
:1013FB00123570EF600302137F12153C123394EF1A
:10140B007003021323900295E06431701A12363088
:10141B00701512150E121523A3E09000F6F012288A
:10142B00F712150E123BD0900295E0643270161233
:10143B003630701112375E9002A1E0FF12152312A5
:10144B002820121517900295E0642D700E1236307D
:10145B0070091214F4122A8E121517900295E0647B
:10146B002E701612363070111214F4122BA1123783
:10147B005E9002A1E0FF123BD0900295E0B4140AFB
:10148B00D2141232807F01123698900295E0B41577
:10149B0005C214123280301447900295E014603567
:1014AB0004703D900296E090014EF0123982E49068
:1014BB0000F2F0E49000F1F09000F1E0FFC394042F
:1014CB00500512153280F19000F2E004F0E0C39465
:1014DB000440E0800B900296E090014EF0123B9599
:0914EB0012153C12328002132399
:1014F40012375E9002A1E0FF123BD712375E9002D2
:1015040097E0FFA3E0FDA3E0FB2212375E9002A167
:10151400E0FF2212375E9002A1E0FF123BD02212BC
:101524003BD7900297E0FFA3E0FDA3E0FB22123635
:081534000B9000F1E004F0222D
:091A1B00E4F5B1F5A975B28322CE
:1039500075A41F75A5E0E4F5A675F2E77590FF75EF
:09396000D40875E10775E242226A
:0A3BAB0075A14075F801E4F5A222AF
:103AB5005389F0438902538EFBE4F58CD28CD2A94D
:013AC50022DE
:1037E000121A1B123BAB123AB5123950123B32126D
:0E37F00038CB121A121232FE123AC60231F90A
:1033640002360234023702350232023301300030B1
:1033740002300231013100310132013301340032B3
:10338400003300340137013601350037003600358B
:0437FE0002120000B3
:1017D600900100E0FE75F00AA42409F582E43401C4
:1017E600F583EFF0EE75F00AA42402F582E43401E5
:1017F600F583227490F090012BE0FEEF75F00AA4B9
:101806002408F582E43401F583EEF09000FEE075DD
:10181600F005A42453F582E43401F583E0FF90003B
:10182600FFE075F00AA42454F582E43400F583E061
:10183600FD7C00229000FFE075F00AA42453F58297
:10184600E43400F583E0FF7E00E50D75F005A42481
:1018560055F582E43401F583E0FD3395E0FCED2F88
:10186600FFEE3C900129F0A3EFF0900129E0FEA3E2
:10187600E0D3947FEE6480948022F090012BE0FE0A
:10188600EF75F00AA42408F582E43401F58322906A
:101896000129A3E0547FA3F0E4900100F022EF7544
:1018A600F005A42455F582E43401F583E0FF339571
:1018B600E0FE229000FFE075F00AA42453F582E4CE
:1018C600340022EF25E025E0243FF582E43402F5DA
:1018D6008322E29000F3F0E804F8E2FF08E2A3CFE7
:1018E600F0A3EFF022900129E4F0A3747FF0229098
:1018F6000100E0FFC3940422E0FF90012BE0FDEF1E
:101906002225E02464F582E43433AF82FE22C3EE5E
:101916006480948022E0FF9000FEE0FE7408A80632
:101926000822740193F2900145E0FCA3E0FDE8046F
:10193600F8ECF208EDF222E4900129F0A3F022F08F
:101946009001007404F022900100E004F02290005F
:10195600FEE0FF7408A8070822EF25E025E02441F1
:10196600F582E43402F5832225E025E02440F58261
:10197600E43402F583229000FEE0FFC3940422754E
:10198600F00AA42451F582E43400F5832225E024EC
:101996006CF582E43433AF822225E02474F582E4C8
:1019A6003433AF8222E0FF90012DE0FEEF4E22E0BD
:1019B600FE54F0649022E0FFAE0D7408A8060822DB
:0719C6009000F374F0F02221
:103A7D007F008F178F147F1B8F188F157F368F192F
:033A8D008F16226F
:103332009000F3EEF0A3EFF0A3ECF0A3EDF0900019
:10334200F574FFF5F01211DB45F060159000F3E41F
:1033520075F0021211DBAFF0FEE4FDFC122DAC8021
:02336200DD226A
:1031F9007B017A02793F9000FAE4F0A37420F0E4AD
:10320900FD123520123A7D7E337F641232377E33C8
:103219007F6C1232377E337F747D047C0012333227
:103229007E337F7C7D067C001233320229CD7D04FA
:063239007C00123332227A
:102DAC00900145ECF0A3EDF0C2A98F828E83E493E1
:102DBC0014601F146034240270568F828E83A81402
:102DCC00121928E5142403F514641B7043751400C0
:102DDC00803E8F828E83A815121928E5152403F5E1
:102DEC00156436702B75151B80268F828E837401AB
:102DFC0093A816F2900145E0FEA3E0FFE804F8EE7C
:102E0C00F208EFF2E5162403F516B45103751636E5
:052E1C00D2A9D21A2228
:0A2FB70090013DECF0A3EDF0AA0735
:102FC100EBD394665017EB75F080A4FDEB25E0FE82
:102FD100E42DFFEE35F0900141F0A3EFF0EA121974
:102FE1000790013DE0FCA3E0FD122DACEB6010EA7F
:102FF100121993FE900141E0FCA3E0FD122DAC906B
:103001000140E0FD600EEA12199FFEED7D0025E012
:04301100FC122DACD4
:013015002298
:052CB00090013AEFF075
:102CB500ED1218BDF583E090013BF090013AE07507
:102CC500F005A42469F582E434011218B090013BA3
:102CD500E0FB7A00EF2BFFEA3EFED3EF12187840B7
:102CE50005747FF080111219145007E490013BF030
:102CF500800590013BEFF090013AE0FF2408F8765B
:102D05003CEF75F005A42467F582E43401F583E012
:102D1500FFED121828122C2A900140EFF090013A8D
:0C2D2500E0FFA3E0FB74FFFDFC022FB7F1
:1036DA001218C97401F00513E513AA127002051233
:1036EA0014FB12195FEAF0A3EBF0EF12196EEDF07A
:0136FA0022AD
:1038B00012195FE0FAA3E0FBC39511EA9510500AD4
:0B38C0008A108B118F0DAF058F0F22B7
:1006A700E49000FEF012197C500EEF1217EBE4F005
:1006B7009000FEE004F080EDE49000FFF09000FF72
:0A06C700E0FFC394104003020C731F
:0F06D100EF121985E0FF90012CF07003020C6A04
:1006E000A37401F09000FFE075F00AA42452F58293
:1006F000E43400F583E090012EF0E49000FEF090E9
:1007000000FEE0FFC394084003020C26EF6003B430
:10071000040DE4F50FF50EF50D74FFF510F511EF6E
:1007200075F005A42451F582E43401F583E0FF90CF
:1007300000FFE0FEEF6E6003020A969000FEE0FF0D
:1007400075F005A42452F582E43401F583E07003CA
:1007500002085590012CE0640160201218C9E07075
:1007600003020A969000FEE012196EE0FE90012E40
:10077000E0FDEE6D6003020A968012E50E60030252
:100780000A969000FEE0FF1218CAE0600B90012D5F
:10079000E0FD1238B0020A96750E0190027F121920
:1007A000AB90027FF09000FEE0FF90012EE0FD1282
:1007B00036DA12197C4003020845A31218BC12183D
:1007C000331218A4EF2DFFEC3E12186940051218E1
:1007D000EB8008121914500312193D1218951218C3
:1007E000F54003020A96EF1217EBE070209001002B
:1007F000E01217EB1217F9122C2A1217D6C083C079
:100800008212191B8002C313D8FC4F802B90010069
:10081000E0FF1217EB1219B570251218861218FE98
:10082000B5051C900100E01217EBC083C0821219BD
:10083000548002C313D8FC4ED082D08312194512C3
:10084000194D0207DE9000FEE024FCFFA3E0FD123C
:100850002CB0020A9690012CE0FC90027FB4030CAD
:10086000E0FE90012DE0F4FDEE5D80031219AB90E7
:10087000027FF012197C400302099CEC64036003C0
:10088000020913A31218BC1218331218A4EF2DFF7B
:10089000EC3E12186940051218EB8008121914502A
:1008A0000312193D1218951218F54003020A96EF2B
:1008B0001217EBE07022900100E01217EB74801227
:1008C00017FB122C2A1217D6C083C08212191B8064
:1008D00002C313D8FC4F802E900100E0FF1217EBEB
:1008E000E0FE54F0648070251218861218FEB505DB
:1008F0001C900100E01217EBC083C08212195480D3
:1009000002C313D8FC4ED082D08312194512194D60
:100910000208A71218B9F583E0FF7E009000FEE000
:1009200012185140051218EB8008121914500312C6
:10093000193D1218951218F54003020A96EF121786
:10094000EBE07020900100E01217EB1217F9122C67
:100950002A1217D6C083C08212191B8002C313D873
:10096000FC4F802B900100E0FF1217EB1219B570BD
:10097000251218861218FEB5051C900100E012170A
:10098000EBC083C0821219548002C313D8FC4ED02E
:0C09900082D08312194512194D0209355E
:10099C00E4900135F0A3F090012CE0B4030AE4904C
:1009AC00012FF0A3F0020A4574FF90012FF0A3F081
:1009BC00900135E4F0A3743C121810122C2AEF2588
:1009CC00E0900131F0A3E4F09000FEE01218A512C3
:1009DC0018B9F583E02FFFE43E900138F0A3EFF057
:1009EC00900138E0FEA3E0FF121877400890013820
:1009FC001218EE800C1219145007E4900138F0A371
:100A0C00F0900138E0FCA3E0FD547F25E090013329
:100A1C00F0A3E4F0D3ED9466EC64809480501A90CB
:100A2C000138E0FEA3E07807C333CE33CED8F9FF0C
:100A3C00900133EE8FF01211C59000FEE024FC9073
:100A4C000137F0900135A3E0FFA3E0FE2408F8A6DF
:100A5C000790012CE06402600FEE12190790012F31
:100A6C00E0FCA3E0FD122DAC90012CE06403601AB5
:100A7C00900137E0121993900133120C76900137E4
:0A0A8C00E012199F900131120C7660
:100A960090012DE025E0F09000FEE0FF6403600881
:100AA600EF64076003020C1D90012CE064017003E3
:100AB600020B70E50F7003020B7090027FE0FFE5FA
:100AC6000FF4FEEF5EF0E50D1218CAE4F0E50DC373
:100AD60094044003020B5D12183A40051218EB808D
:100AE60008121914500312193D1218951218F540E0
:100AF60003020C1DEF1217EBE07025900100E012C7
:100B060017EB7480121880EEF0E50D121815122CF2
:100B16002A1217D61219BC8002C313D8FC4F802E96
:100B2600900100E0FF1217EBE0FE54F064807021A4
:100B36001218861218FEB50518900100E01217EB80
:100B4600AF0D7408A807088002C313D8FC4E12190B
:100B56004512194D020AF2E50D24FCFFE49001400E
:100B6600F0FBFDFC122FB7020C1DE50E6003020C14
:100B76001DE50F7003020C1D90027FE0450FF090FB
:100B8600012EE0FDAF0D1236DAE50DC39404507A5E
:100B960012183A40051218EB800812191450031265
:100BA600193D1218951218F5506DEF1217EBE070FB
:100BB60025900100E01217EB7490121880EEF0E514
:100BC6000D121815122C2A1217D61219BC8002C340
:100BD60013D8FC4F802B900100E0FF1217EB12197F
:100BE600B570211218861218FEB50518900100E09E
:100BF6001217EBAF0D7408A807088002C313D8FCC0
:100C06004E12194512194D020BABE50D24FCFF904F
:100C160000FFE0FD122CB09000FEE004F00206FF9B
:100C2600E4900100F0900100E0FE1217EBE0FF6097
:100C36002AEE121887E0FD900100E075F00AA42460
:100C460009F582E43401F583E0FB1234A690010035
:100C5600E01217EBE4F012194D80CA9000FFE01283
:040C66001985E4F018
:0C0C6A009000FFE004F00206C40232809B
:0A0C7600FEE0FCA3E0FD122DAC220D
:1029CD00201A03022A6DC21AE514B5170EE515B5C6
:0B29DD001809E51665197003022A6D49
:1029E800C283E516B519051219C68011A81912185F
:1029F800D8E5192403F519B45103751936122A6E4E
:102A0800122A87E515B518051219C68011A81812DB
:102A180018D8E5182403F518B4360375181B122ABC
:102A28006E122A87E514B517051219C68011A81762
:102A38001218D8E5172403F517B41B03751700E41B
:102A4800FF123BC89000F3E0FF123BC89000F4E08F
:102A5800FF123BC89000F4A3E0FF123BC8121A090A
:022A6800D28317
:102A6A000229D522E4FF123BC89000F3E0FF123B93
:102A7A00C89000F4E0FF123BC89000F422A3E0FFE4
:042A8A00123BC82211
:1039E30074082FF8E6600F16E6700BEF1219077DC7
:0739F300007C80122DAC22C4
:031A06000219CDF5
:1019CD00C0E0C083C082C0D075D000C000C003C0CD
:0719DD0004C005C006C007AD
:0C19E400E4FBAF031239E30BEBB404F694
:1019F000D007D006D005D004D003D000D0D0D082FC
:051A0000D083D0E032AC
:103AE80000FF0100010000FFFF0000010001FF00CE
:0738020042027D0000C11726
:0F3AF800E56E856F838570822290014B02120D5F
:052E8F0090014AEFF084
:102E9400E56D2401FFE4356CFAA9077B01A3121246
:102EA4002D123B0174019002946B7008E9658270E5
:102EB40003EA6583700C7B017A02798090014B12DE
:102EC400122D123B01123AF86B7008E96582700307
:102ED400EA6583601990014AE0856D82856C83F010
:0E2EE400123B01AF018A6C8F6D90014AE0F045
:012EF20022BD
:0E3B1600EB5F6009ED5B6005AF03122E8F229E
:0D3B320075BC4475E8C075BA1F75D1082236
:10311A0053E6EFAA6CA96D7B01123AF86401700AB2
:10312A00E56D65827004E56C65837003FF802B781A
:10313A006EE475F0011211FD1210DBFF74019002AA
:10314A0094656E700AE57065827004E56F65837038
:0D315A0009756E01756F0275708043E610F7
:013167002245
:1035700053E6EF123AF86401700AE56D6582700453
:10358000E56C65837003FF800AAB6EAA6FA97012A9
:0635900010DBFF43E61012
:013596002212
:10365300EFD394B840047E108016EFD394784004DF
:103663007E04800CEFD3945040047E018002E4FE7C
:02367300AF06A0
:013675002232
:031A24000221F7A5
:1021F700C0E0C0F0C083C082C0D075D000C001C0AD
:0F22070002C003C005C006C00720DF030222A4E7
:10221600900148E5BEF0D2ECA216B3921630160D28
:1022260075BB04E0FF1236538F6A0222A275BB0308
:10223600900148E0FF123653EF25E0426AE56A65F1
:10224600746012E56A6574900147F0543F60037547
:102256007203856A74E57260431572E572703DE536
:1022660073656A900147F090027DE07002A3E0601A
:1022760006E56A7002D2177B011223197B02AD6A4A
:10228600123B167B041223197B081223297B10129A
:0E22960023297B20AD6A123B16856A73C2DFD6
:0622A40020D80330D958D8
:1022AA00900147E590F0C2D9C2D8E0FD65715403A8
:1022BA006046E57175F004A47E00540CFFED5403EA
:1022CA00FDEF4D24E8F582EE343AF583E493FF906E
:1022DA000148F0A3E56BF0EF256BF56BE0656B3019
:1022EA00E110900148E0B401047F0980027F0A12DC
:0822FA002E8F900147E0F57101
:10230200D007D006D005D003D002D001D0D0D082E1
:10231200D083D0F0D0E032900147E0FFAD6A123BAB
:1023220016900147E0FF22AD6A123B16900147E08A
:02233200FF2288
:0C3B590075DA3175DB3175D989D2DE22B6
:1038CB00123B597B017A0279808B6E8A6F89708AE1
:0B38DB006C896DE490027FF0023280E7
:061A0900E5A120E7FB222D
:083BC800E5A120E7FB8FA32219
:103280007D017C00E4FB900237E0FFEBC39F500A16
:10329000ED25E0FDEC33FC0B80EC301404EC4440F5
:1032A000FCC2AFD28390027FE0F4FF123BC8ECF483
:0F32B000FF123BC8EDF4FF123BC8121A09D2AF50
:0132BF0022EC
:1036FB00A2AFE433FCC2AF758F0175B7A575B7F1F7
:10370B008F828E83EDF0E4F58FAF04EF24FF92AF41
:01371B00228B
:101F6400000102040810000003041800000000002F
:101F74001F00000000001804030000000010080403
:101F840002010000040A0A11110000010102021CEE
:101F940000001C02020101000010100808070000E4
:101FA4000708081010000018180018180000181866
:101FB40003181800008040C020A060E0109050D0AA
:101FC40030B070F0088848C828A868E8189858D82D
:101FD40038B878F8048444C424A464E4149454D42D
:101FE40034B474F40C8C4CCC2CAC6CEC1C9C5CDCCD
:101FF4003CBC7CFC028242C222A262E2129252D215
:1020040032B272F20A8A4ACA2AAA6AEA1A9A5ADACC
:102014003ABA7AFA068646C626A666E6169656D6CC
:1020240036B676F60E8E4ECE2EAE6EEE1E9E5EDE6C
:102034003EBE7EFE018141C121A161E1119151D1D8
:1020440031B171F1098949C929A969E9199959D99C
:1020540039B979F9058545C525A565E5159555D59C
:1020640035B575F50D8D4DCD2DAD6DED1D9D5DDD3C
:102074003DBD7DFD038343C323A363E3139353D384
:1020840033B373F30B8B4BCB2BAB6BEB1B9B5BDB3C
:102094003BBB7BFB078747C727A767E7179757D73C
:1020A40037B777F70F8F4FCF2FAF6FEF1F9F5FDFDC
:0420B4003FBF7FFFAC
:0D3B24007FC87E00EF1F70011EEF4E70F78E
:013B31002271
:103AC6007F38123A557F06123A557D0EE4FF023BC7
:013AD600658A
:103A550090011DEFF012399BEF20E7F990011DE071
:043A6500FF0239B370
:10399B0075A0FFC296D295D2977F14DFFEAFA0EF32
:0739AB00901FB893FFC297C3
:0139B20022F2
:053BF0007F01023A55BF
:1039B300EF901FB893F5A0123B24C296C295D297FD
:0839C300123B24C297023B24D1
:10371C00EF3395E0FE74B82FF582741F3EF583E409
:10372C0093F5A0C295D297D296123B24C297023B36
:01373C002468
:0C3B65009002A2E05FF04DFFF0023A5524
:0B396900E475F0011212161210DBFFD3
:0E397400AE0712399BEF20E7F9AF0602371CB1
:10391C0090011D12122D90011D12120D1210DB6060
:0A392C000890011D12396980ED2298
:1034F80090011712122D123BF0E4FDFF123B719060
:10350800011712120D12391CE4FD7F01123B719054
:08351800011A12120D02391C08
:0C3B7100EF75F040A42D2480FF023A55AF
:08316800900117EFF0A3EDF058
:10317000E075F008A42440FF123A55900117E0547E
:103180007F75F007A42464F9741F35F0FA7BFF9073
:10319000011912122D900118E0900117F07D07AF70
:1031A000051DEF600890011912396980F2E4FF02F1
:0231B000397470
:053520009000F9EDF040
:10352500AE02AF019000FA74FFF5F01211DB45F021
:1035350060109000F9E08F828E83F00FBF00010EBE
:0235450080E222
:013547002261
:0D3B3F00AE05AD07AF06AB077F0A0234A646
:103A900090011CEFF012375E90011CE0FF1230160F
:033AA000023B895D
:053BF5007F02023A907E
:06339400123BDEEF602792
:10339A009000F37402F0A37494F01234CF9000F307
:1033AA00E475F0011211DB85F082F583EFF0123B30
:0733BA00E4EF70E67F012241
:0333C1007F002268
:10381C009000F3EFF0A3EDF012375E9000F3E0FFB1
:0E382C001230169000F4E0FF123016023B89B5
:1034A60090013AEFF0A3EDF0A3EBF012375E900136
:1034B6003AE0FF12301690013BE0FF123016900101
:0934C6003CE0FF123016023B89C4
:073BD000AD077F2F02381C36
:073BD700AD077F3002381C2E
:1039CB000002000200020002000100010002603050
:0839DB002018100C080604037B
:0E380900C10E410215004101DF004101E00047
:102334003CFA7B019000F4E0FF3395E0FEEF25E0EA
:10234400FFEE33FE22C374809DFDE49CFC74C12D1A
:10235400FD74FF3CC3648094802290337C75F0024A
:102364001211F1AF82AE832275F00AA42453F582D0
:10237400E43400F583E5822FF582E5833EF583227C
:10238400EF75F005A42479F582E43401F583E022A5
:10239400EB9039D993FD3395E0FC9001E2E024FF02
:1023A400FF9001E1E034FFFE2275F00AA42451F508
:1023B40082E43400F58322740D2FF58274023EF515
:1023C40083E02275F005A4247BF582E43401F583CF
:1023D400E0FE2275F00AA42452F582E43400F58369
:1023E400EFF02275F005A4247AF582E43401F58334
:1023F400E022E07D0025E0FC9001E4E0FB22900077
:10240400F5E0FD74017E00A8050822E0FF9000F9C4
:10241400E0FE7408A80608223CFAE92FF9EA3EA86F
:1024240001FC7D012275F00AA42454F582E43400F1
:10243400229001E4E075F00AA4FDACF0227E007F56
:10244400021210B59000F4E0229001ECE0FF90013C
:03245400E4E0229F
:1035E5007B017A0079519000FAE4F0A374A0F0E42D
:1035F500FD123520E490027FF0C20DC20A9001E170
:06360500F0A3F0C20E224A
:093BBF001235E51231F9D2092298
:102C2A00EF1212422C74012C50022C6B032C4D040F
:102C3A002C7F052C62062C55072C90082C9D090028
:102C4A00002CAD022CA87D50022CAD12235150024B
:102C5A00E4FDED25E0FD80461223515030E4FD806D
:102C6A002CC374809DFDE49C8001ECA2E713ED1354
:102C7A00243CFD802ED3ED943FEC64809480400484
:102C8A00747F9DFD80071223495002E4FDED25E083
:102C9A00FD80101223495002E4FDED25E0FDC374C6
:062CAA00809DFDAF052234
:10360B007408A807088002C313D8FC44B0FEEF75FA
:10361B00F005A42454F582E43401F583E0FBAF06F6
:05362B007D1F0234A622
:0E32C000AB05AA0712239412118FED4C702E4D
:1032CE0012239412113A9000F6EEF0A3EFF0900054
:1032DE00F6E475F0011211C50AEAFD7C009000F6C5
:0E32EE00E0FEA3E0FF12113AED4C7002D32275
:0232FC00C322EB
:10245700E49000F5F09000F5E0FFC3940640030216
:10246700252C122384641060030225239000F5E0D5
:102477001223E7FE12254D501A9000F5E012235E55
:1024870074FF12252D7401A806088002C333D8FCF7
:102497004F80291224028005C333CE33CED8F9FFEB
:1024A7009001DFE0FBEF5B6017ED12235EE412257E
:1024B7002DE4A806088002C333D8FC5F9001DFF043
:1024C7009000F5E01223C712254D501D9000F5E04E
:1024D70090338812236174FF12253D7401A8060802
:1024E7008002C333D8FC4F802F1224028005C333E8
:1024F700CE33CED8F9FF9001E0E0FBEF5B601D75AE
:10250700F002ED903388122364E412253DE4A80617
:10251700088002C333D8FC5F9001E0F09000F5E03B
:0525270004F002245C39
:10252C0022FDFC122DAC9001DFE0FF9000F5E0FEE7
:10253C0022FDFC122DAC9001E0E0FF9000F5E0FED6
:0D254C0022C4540FFFEE540FFD1232C022C6
:0E1C08009000F5EFF0A3ECF0A3EDF0A3EBF0ED
:101C16009000FA74B0F0A374E0F0E49000F9F0904C
:101C260000F9E0FFC39404504BEF75F005A424516E
:101C3600F582E43401F583E0FF9000F8E0FEEF6EF4
:101C4600702A9000F5E070139000FB12240F8002BA
:101C5600C313D8FC4F9000FBF080119000FA1224B9
:101C66000F8002C313D8FC5F9000FAF09000F9E0F1
:101C760004F080ABE49000F9F09000F9E0FFC39423
:101C860006505CEF1223E7FF9000F5E0FEEF6E7062
:101C9600199000F9E0FF122385FE9000F8E0FDEEB2
:101CA600B50507EF12235E121DB49000F9E0FF128E
:101CB60023C79000F5E0FDEE6D701B122384FF90A4
:101CC60000F8E0FEEFB5060EA3E075F0029033884B
:101CD600122364121DB49000F9E004F0021C7F90F8
:101CE60000FAE0FF540F600C9000F5E0FDA3A3E0BE
:101CF600FB1234A69000FBE0FF540F6023C0079050
:101D060000F6E0FAA3E0FBAE027802CEC313CE13D0
:101D1600D8F9547FFDEAC313547FFBD0071234A6CB
:101D26009000F5E064426003021DB39000F8E09075
:101D36000215F0A20A920DC39000F6E09480506B53
:051D4600C20A300D6827
:061D4B009000FC7403F09F
:101D51009000FD7403F09000FDE0FFC36480948067
:101D61004023EF12233D900215E0FD122429122396
:101D710077E4F01223BBFCED12236CECF09000FD34
:101D8100E014F080D1900215E0FD1223AD7403F050
:101D91009000FC12233B1223BBFFED1223D7120646
:011DA100A79A
:0F1DA2009000FCE014F0E0C36480948050A12214
:021DB100D20A54
:0D1DB300229000F6E0FCA3E0FD122DAC2212
:101A2700EF1212421AB2801A4A901B9EA01BA8B04E
:101A37001B80E01BE1F81BB8FA1BD8FB1BCFFC008F
:091A4700001C079001EDE0606253
:101A50009000F47402F01224352453F97400122318
:101A600034E92FF9EA3EFAC002C00174552DF97429
:101A70000012241CD001D00212244114F0E0C364EF
:101A800080948050D112244DFE75F00AA42453F5A1
:101A900082E43400F583EFF09001EDE0FDEE1224D6
:101AA00029F583EDF0EE1223AD7401F0D209EE02B8
:021AB0001B7A9F
:101AB200300A529000F47402F09000F4E0FFC36424
:101AC2008094804034EF12233D1223BBFD740F2F0C
:101AD200F58274023EF583EDF0740E2FF5827402E6
:101AE2003EF583E0FD74102FF58274023EF583ED1E
:101AF200F09000F4E014F080C09001ECE090020D50
:101B0200F0E4A3F022E49000F4F09000F4E0FFC3CC
:101B120064809484505FEF12233D9001E4E012232D
:101B22006CE0FF9001ECE0FEEF6E70409000F4E09C
:101B3200C36480948350291224352455F974001209
:101B42002334E92FF9EA3EFAC002C00174532DF999
:101B5200740012241CD001D00212244104F080CC63
:101B62009001E4E01223AD7403F0D2099000F4E096
:0E1B720004F0021B0C12244D1223D7021C0794
:101B80009001ECE075F004A4FDA3E025E0FEE42D57
:101B9000FFEE35F0FEAD071223FBE4FF8015900148
:101BA000ED1223F67F01800B9001ECE02402FFA3ED
:101BB0001223F6121C08804FD20EE49001DFF0A32E
:101BC000F07FFA123A90E49001E1F0A3F080387FC0
:101BD000FC123A90C20E802F7FFB123A90D20E80F8
:101BE00026300E237FF8123A909001E1E475F0015F
:101BF0001211DBFEE4B5F00CEEB403089001E1E451
:071C0000F0A304F0122457C9
:011C070022BA
:102E2100AE07EF70089001E5F0A3F08059EE54F081
:102E31009001E3F0EE540FA3F0EEC394F04026901E
:102E410001E3EEF0B4F00BE49001E9F09001E7F05A
:102E5100A3F0EEC394F85005E49001EAF09001E488
:102E610074FFF080219001EAEEF0C4540F25E024B4
:102E7100BBF582E43439F583E493FF740193900147
:0E2E8100E5CFF0A3EFF0E49001E7F0A3F0221C
:102D31009000F3EFF030E727E0FFF4606DEF64F807
:102D4100600EEF64FA6009EF64FC6004EFB4FB030A
:102D5100021A279000F3E0FFC394F7504D8048908A
:102D610001E5E07002A3E060419000F3E0FF900113
:102D7100E9E02FF09001E7E475F0011211DBFC743A
:102D8100EC25F0F58274013CF583EFF09001E574D8
:102D9100FFF5F01211C545F070109001E3E0FF124C
:0B2DA1001A279001EAE0FF122E212209
:011A0500FFE1
:10265800E475F0010211C5E0FCA3E0FFECFDE49095
:10266800010AF0D2007BA62290014EE075F046A444
:10267800FF900150E02FFF90014FE035F0229001CC
:10268800037B017A017951E4F0A37446F022EDFF4F
:10269800AD04EDCFF0A3EFF0C2AF43C15E90014EA1
:1026A800740FF022EF75F005A42454F582E4340188
:1026B800F5837432F022FE9000F9E09FEE6480F812
:1026C8009000F8E064809822E0FCA3E0FFECFD2293
:1026D800E024FFFEE434FF9000F8F0A3CEF022EEF1
:1026E800F0A3EFF0A312122DA2AFE43322A42451D9
:1026F800F582E43401F58374FFF022EF9001507500
:10270800F046A4FFE022EBF0AC07A2AFE433A3F05D
:1027180022F0C2AF43C15E2274FFF5F01211DB450F
:10272800F022F583E4F0EF75F005A4222FFEEC35D6
:06273800F0F0A3CEF02238
:03323F009000FEFE
:103242001226E79001051227199001031227206028
:10325200219000FE12265F12273E90010012120DED
:10326200EF1211169000FE122658900101122658F4
:0D32720080D71232FE900105E024FF92AFDC
:01327F00222C
:0330C8009000FE77
:1030CB001226E790010512271990010312272060A1
:1030DB003290010012120D1210DBFC900106F090E1
:1030EB0000FEE0FAA3E0FFEAFD90010AECF0C2005B
:1030FB007BA612273E9001011226589000FE122645
:0E310B005880C61232FE900105E024FF92AFFC
:013119002293
:102B18009000FA122689E4FD123520E49000F3F0C3
:102B28009000F3E0FFC3940E5045EFC39408EF758F
:102B3800F005502C1226F51226ACEF75F005A424EA
:102B480053F582E4340112272A2452F582E4340131
:102B580012272A2455F582E43401F583E4F0800332
:102B68001226F51226AC9000F3E004F0022B28E4BC
:102B78009000F3F09000F3E0FFC3941E501AEF1298
:102B88002674FE9000F4F0A3EFF01226861230C8E7
:082B98009000F3E004F080DC82
:012BA0002212
:0C3B7D00201808301405123BF5D2182265
:10373D00E490014FF0A3F0901A0593600C122B1832
:10374D007E1A7F05E4FD1236FBE490014EF0C2189F
:01375D002249
:10398200123BBF122670FE7B017A0179519001032E
:0839920012268F12323FC21809
:01399A00220A
:0A3BB500122670FE1226860230C8A8
:0B3B9500123BBF123BB5C2180235E521
:0A28F7009000F4EDF09000F3EFF014
:10290100D39B402E1226D8EB149000F7F09000F4E0
:10291100E024FFFFE434FFD31226BE504B12296A94
:102921001230C89000F81226589000F7E004F00227
:10293100290E9000F41226D89000F6E014A3F0902E
:1029410000F3E024FFFFE434FFC31226BE40191256
:10295100296A1230C89000F874FFF5F01211C59081
:0829610000F7E014F002294028
:10296900229000F7E075F046A4FF90014FE0FAA32A
:10297900E0FB2FFEEA35F09000FAF0A3CEF09000CC
:10298900F8E0FEA3E0FF7C007D46121128EB2FFF43
:10299900EA3EFE9000FCF0A3EFF07B007A00792478
:1029A900900103E4F0A37446F012323F9000FAE07C
:1029B900FEA3E0FF7B007A007924900103E4F0A3F1
:0429C9007446F0223E
:0E3B0700E4FFFE0FBF00010EBE13F8BF88F5ED
:013B1500228D
:052820009000F3EDF053
:10282500A2AFE4339000FE122719EF149000FAF0DE
:10283500EB14A3F09000F3E014FF9000FAE0FED350
:102845009F40030228DEEE90014F122707FCA3E00C
:10285500FD9000F61227349000FBE075F046A4FFCA
:10286500ED9000F8122734E49000F4F0A3F0900006
:10287500F612265F12273E9000FCEFF0123B079000
:1028850000F812265F12273E9000FDEFF0123B077D
:102895009000F81226D09000FC1228EA123B07900F
:1028A50000F61226D09000FD1228EA9000F81226B4
:1028B500589000F61226589000F4122658C390003E
:1028C500F5E094469000F4E0940040A29000FAE010
:1028D50004F0A3E004F00228391232FE9000FEE075
:0428E50024FF92AF8B
:0E28E90022E090010AF0C2007BA612273E22D8
:032BA1009000F3AE
:102BA40012270E9000F712269690014EE0FFC39470
:102BB4001E50671227032FFE12267F9000F9F0A300
:102BC400CEF0E49000F5F0A3F09000F71226D09038
:102BD40000F3E0FBE490010AF0D20012273E9001DA
:102BE4000AEFF09000F91226D0C2007BA612273E0D
:102BF4009000F91226589000F71226589000F5120A
:102C04002658C39000F6E094469000F5E094004006
:102C1400B890014EE004F0022BAD1232FE9000F4A5
:052C2400E024FF92AF67
:012C29002288
:032A8E009000F3C2
:102A910012270E9000F812269690014EE0FFC39483
:102AA1001E50681227032FFE12267F9000FAF0A312
:102AB100CEF0E49000F6F0A3F09000FA12265F1237
:102AC100273E9000F5EFF0FC9000F8E0FAA3E0FF5C
:102AD100EAFD9000F3E0FB90010AECF0C20012273E
:102AE1003E9000F81226589000FA1226589000F6EF
:102AF100122658C39000F7E094469000F6E0940047
:102B010040B790014EE004F0022A9A1232FE900082
:062B1100F4E024FF92AF86
:012B1700229B
:103A6900EFFD90010CE0FB3395E0FAC3EB9D748008
:043A7900F86A98222D
:08273E00900107EFF0A3EDF09C
:10274600A2009204C206201BFDD21B90010BEBF0E7
:10275600C201D202D2057F01C2C4C207D2C530C0AF
:10276600FDE5C054F02480607624C0601B24E06040
:102776000302280590010BE0F5C2A201E43342C230
:10278600C2C5E4A3F002280730C149300707D2C505
:10279600C20702280730020CC202D203900108E0E9
:1027A600F5C2805D300311C203900107E0F5C23027
:1027B600044FD207D2018049200146123A69500ED1
:1027C60090010AE0F5C290010CE004F08033D2C417
:1027D600C21B802D300504D2C58026D20680221267
:1027E6003A69500CA3E5C2F090010CE004F0D2C1A6
:1027F60090010CE0B5070AC21BC2C1D2C48002D246
:102806000630060853C0BF43C040C21BC2C0301BBF
:092816000302276490010DE0FFAC
:01281F002296
:0D3B4C007E027F5F8E778F788E758F7622D8
:103A3F0053890F438920758E01758DCFD28E75985E
:063A4F0010D2ACC2BC2243
:061A1200123B4C023A3FBA
:013BFA0022A8
:103AA300E57665787004E575657760037F01227FAD
:023AB3000022EF
:103676000578E578AE777002057714F5828E83E0DB
:10368600FF747DB5780B7402B57706757702757889
:013696005FD4
:013697002210
:031A0F000231B2EF
:1031B200C0E0C083C082C0D030982EC2988576828B
:1031C200857583E599F00576E57670020575B47D1F
:1031D2000BE575B4020675750275765FE576B5780E
:1031E20008E575B57703123BFA309902C299D0D03F
:0731F200D082D083D0E0324F
:02381700C111DD
:103073009001A1E475F0011211DB85F082F5832242
:1030830090019DE0FFA3E0CF900199F0A3EFF02220
:103093009001A17401F0A374B7F022900199E47533
:1030A300F0011211C57E017FDF900199E022E0FE5D
:1030B300A3E0FF900199E0FCA3E0FD22EE90019DC7
:0530C300F0A3EFF02274
:0B3BA000D2CB438E2075CBE8D2CA22A6
:103AD70075C102E4F5C2F5C053C17F43C180023B03
:013AE700A03E
:1032FE007E017FA390019BEEF0A3EFF090019FEE75
:10330E00F0A3EFF0900197EEF0A3EFF07E017FB700
:10331E001230BF9001A1EEF0A3EFF0EE12308BC28F
:04332E0010023AD778
:1035970090019F123076EFF090019F123076EDF098
:1035A70090019FE0B4010FA3E0B4B70A90019F74A4
:0735B70001F0A374A3F02250
:0C3B8900E5C120E5FBC210C2C4D2C52279
:1030160020102FD21012307374FFF07C017DDF90E8
:1030260001A1E0B50408A3E0B50503123093123000
:1030360073E4F09001A1E0B50408A3E0B50503121E
:103046003093123073E4F09001A1E0B40108A3E0DC
:10305600B4DF03123093123073EFF09001A1E0B4A5
:0D3066000108A3E0B4DF031230937F0122C4
:10344F0090019BE0FCA3E0FD900197E0B50408A379
:10345F00E0B505037F002290019BE0FCA3E0F5821D
:0C346F008C83E0B507037F01227F002260
:1034CF0090019BE475F0011211C590019B123076AB
:1034DF00E0FF90019BE0B4010FA3E0B4B70A9001A5
:0834EF009B7401F0A374A3F02B
:0134F70022B2
:063BDE007FFF12344F22AC
:063BE400E4FF12344F2241
:031A1800021DC0EC
:101DC000C0E0C0F0C083C082C0D075D000C000C0E9
:101DD00004C005C006C007E5C054FE1212421F2E03
:101DE000081F2E0A1F440C1F440E1F07101F071246
:101DF0001F23141F23161EFA1C1EFA1E1EF6241E75
:101E0000F6261EAA281EAA2A1EC72C1EC72E1E4C46
:101E1000C01E56C21E1EE01E1EE200001F4DC2C59F
:101E200012309EB5060BA3E0B5070690019912305B
:101E300096900199123076E0F5C2900199E06E70AB
:101E400003A3E06F6003021F4D021EA1123083D274
:101E5000C4D2C5021F4D9001A11230B1B5070EECDE
:101E6000B5060A1230BFC2C5D2C4021F4D8D828C86
:101E700083E0B4FF03021F4912309EB5060BA3E0B6
:101E8000B50706900199123096900199123076E0CC
:101E9000F5C2900199E06E7003A3E06F6003021F2A
:101EA0004D900199123096021F4DE5C260379002A5
:101EB000A1E065C2602FC2C4C2C5C2C1C2129002F5
:101EC0009E7401F0021F4D123083C2C5D211E5C2CB
:101ED00060139002A1E065C2600BC2C4C2C5C2C15A
:101EE000C212021F4DADC27FFF123597C2C4C2C5D8
:101EF000D2C1D2128057D2C58053900199E0FFA37E
:101F0000E0CF1230C0804690019FE0FFA3E0900137
:101F100097CFF0A3EFF0C2C4C2C1301130D2C5C216
:101F200011802A123083C2C4C2C1D2C5801FC2C46C
:101F3000C2C5201204C2C18014ADC2E4FF1235979D
:101F4000D2C18009123083C2C1C2C4D2C5C2C0D0BE
:101F500007D006D005D004D000D0D0D082D083D016
:041F6000F0D0E032AB
:10375E0090019D1230B1B507F7ECB506F39001A1BB
:10376E00E0FEA3E0FFEDB507E7ECB506E320C5E00C
:01377E002228
:1020B800202020496E697469616C697A696E6720AD
:1020C8002020200020004D6F6E6F00506F6C79004B
:1020D8002050570041667400253364006275733AD6
:1020E80025632043683A25326420257300547225FD
:1020F800632532642046743A416E20566C3A256353
:1021080000547225632532642025732532642056D5
:102118006C3A25630046740046743A0058706F7331
:10212800653A252B3364202056656C3A25630042B6
:1021380075733A2563204368616E3A436C6F636B2D
:10214800004469763A2025642F252D3264203A20F0
:1021580025642F252D3264004275733A2563204388
:1021680068616E6E656C3A25326400436E74726CF9
:102178006C72733A00000AFF3876000CFF3548018C
:1021880004FF33C4010AFF347B010FFF3A11000A30
:10219800FF3876000CFF35480108FF33C4010FFFF4
:1021A8003A11000FFF3893010BFF3936010FFF3A40
:1021B80028000FFF38930105FF383A0107FF37A0C1
:1021C800010CFF3858010EFF37C0414243444546D1
:1021D80047484A4B4C4D4E5000FF20CEFF20D3FFBE
:0F21E80020D8FF20DC0102030406080C10182089
:02381900C19458
:10255900900237E0FE75F005A42451F582E43401B8
:10256900F583E02FF0EE75F005A42451F582E434EB
:1025790001F58322EF540FC454F0FF900237E07540
:10258900F005A422EE75F005A42455F582E4340182
:10259900F58322EF75F005A42453F582E43401F59F
:1025A90083E0222452F582E43401F583E0227BFFA3
:1025B90090011E02122D2453F9740135F0FA7B01A2
:1025C900E0FD9001202290021612120D0210DB90FC
:1025D9000237E0FF9021D293900121F0222452F991
:1025E900740135F0FA7B01E0FD2275F005A4241F82
:1025F900F582E43402F5832275F005A4241DF582E1
:10260900E43402F5832275F005A4241EF582E4342E
:1026190002F58322C4540F2401FCE433F0A3CCF067
:1026290022EF3395E0900122F0A3EF22FE3395E0EB
:10263900F0A3CE22900237E0FF75F005A422E0FF57
:0F2649005480FD3395E04D227B017A0179042204
:1033F400E490023DF0A3F090023BF0A3F090023978
:10340400F0A3F0900238F0900237F07BFF7A207935
:0E341400CC90011A12122D7A2079B80234F8E9
:063BEA00E4900219F02234
:102EF300900117EEF0A3EFF0AF051DEF60539001C3
:102F030017E0FEA3E0F5828E83A3A312123690028C
:102F130019E0FF1225F312122D900117E0FAA3E036
:102F2300FBF5828A83E493FEEF122601EEF08B8297
:102F33008A83740193FF900219E012260FEFF09039
:102F43000219E004F0900117E475F0051211C58031
:022F5300A722B3
:10377F001225CFFE122601E0FFEE12260FE0FD12FA
:10378F003B711225CF1225F312120D90021A02125D
:01379F002DFC
:1039FA001225CF7007900219E012111690021612C2
:073A0A00120D74FF0210F41D
:1038E60090021612120D74011210F41225CFFF90D9
:0B38F6000219E0B50704E412111622CD
:10342200ED1210F41210DBFF3395E0FE900120E064
:10343200FDD3EF9D7480F86E984003E0800B12106C
:0D344200DBC3648094805004E41211162254
:1039010090011BEFF0AF037B017A01791B9001203D
:0B391100EFF012342290011BE0FF22B7
:10387600122559E0FFB4FE0812256E740FF0800A77
:0D388600EFB4100612256E74FFF0023B7DBA
:10389300122559E0FFB4FE0812256E7410F0800A59
:0D38A300EFB4110612256E74FFF0023B7D9C
:1035480090011BEFF012258490011B1225E69002D2
:1035580037E0C3940450047F0280027F0190012069
:08356800EFF0123422023B7D5A
:1033C400900237E0FE12258EE02FF012258DE0FFEB
:1033D400D3648094B0400812258D7430F0800EC3FD
:1033E400EF64809450500612258D74D0F0023B7D1A
:10347B0090011BEFF01225842454F9740135F0FAF6
:10348B007B0190011BE0FD9001207463F01234224C
:0B349B00123B7D900237E0FF02360B71
:103A110090011BEFF012258490011B1225BF740940
:073A2100F0123422023B7D8C
:10383A00AE071225841225ACC4540FFFAD067B07D0
:0E384A0012390112257D1225AC540F4FF022C9
:1037A000AE071225841225AC540FFFAD067B09121B
:1037B0003901EF540F1225831225AC54F04FF0223B
:10385800AE071225841225A1C4540FFFAD067B07BD
:0E38680012390112257D1225A1540F4FF022B6
:1037C000AE071225841225A1540FFFAD067B091206
:1037D0003901EF540F1225831225A154F04FF02226
:1039360090011BEFF012258490011B1225E69001E1
:0A394600207482F0123422023B7D4F
:103A280090011BEFF012258490011B1225BF7482B0
:073A3800F0123422023B7D75
:102F550090011712122D90011AEDF0C39402503012
:102F6500E075F003A424E7F582E43421F583121219
:102F750036C003C002C00190011712120DA801ACA2
:102F850002AD03D001D002D0037E007F030210B54D
:102F95007A2079E01225B790011AE024FEFEE43488
:102FA500FF900121F0A3CEF090011712120D120C23
:022FB500E52213
:10153C00123BEA900237E0FFC3940840030216BF47
:10154C0012259CFF7D011231687A2079E41225B7AF
:10155C001225D8EF12256FE02401FF900122E4F050
:10156C00A3EFF01225841225AC75F003A424E1F549
:10157C0082E43421F58312123690012412122D12BA
:10158C0017CC900237E0FFC394044003021694EF8B
:10159C0012258EE07D0230E7047F0B80027F0A1259
:0215AC003168A4
:1015AE0012263D2454F582E43401F583E0FD7C00DF
:1015BE00900115ECF0A3EDF06432702C7BFF7A20D5
:1015CE0079F51225B99001217402F0EF12258E12D1
:1015DE0026476006EFF404FF800812258412259238
:1015EE00E0FF12262A02167F900115E0FEA3E0FF0F
:1015FE00D39432EE64809480400A90011574FF7586
:10160E00F0CE8013C3EF9432EE64809480500B9032
:10161E00011574FF75F0CF1211C57BFF7A21790980
:10162E001225B99001217402F0122584122592120E
:10163E0026476006EFF404FF8008122584122592D7
:10164E00E0FF12262AF0900115E0FEA3E0FFC394FE
:10165E00F7EE6480947F7BFF50067A21791D80041B
:10166E007A21792090012412122D900127EEF0A3F9
:04167E00EF1217BE92
:101682007E217F7D7D05122EF37B017A027938025D
:1016920017A57BFF7A2179241225B91225841225F8
:1016A20092E09001211226351217BE7E217F967D8F
:1016B20004122EF37B017A0279390217A5900237C0
:1016C200E012256FE02401FFE433EF64117BFF7029
:1016D200697A2179371225B9900237E01225DD1295
:1016E20017CC7BFF7A2179491225B912263D1225A2
:1016F200ACFE90012112261DEE540F9021ED93FCB9
:101702003395E0900123F0A3CCF012259CFF9001C9
:101712002512261DEF540F9021ED939001271226DA
:1017220035F0122651120CE57E217FB97D05122E6D
:10173200F37B017A02793D0217A57A21796012259D
:10174200B91225D8EF12256FE02401FFE43390018E
:1017520022E4F0A3EFF07B017A0079F3120CE57B2F
:10176200FF7A2179731225B9122651120CE512253E
:10177200841225ACFD7B017A01790D122F551225B9
:10178200841225A1FD7B017A017911122F55900156
:1017920010743AF07E217FAA7D03122EF37B017A28
:1017A20002793B90021612122D12265190011A1242
:0C17B200122D7A0079F31234F802377F10
:1017BE00F0A37401F0FB7A017904120CE5227B018F
:0817CE007A0079F3120CE52208
:03000000020600F5
:03000300021A03DB
:03000B00021A06D0
:03001300021A09C5
:03001B00021A0CBA
:03002300021A0FAF
:03002B00021A12A4
:03003300021A1599
:03003B00021A188E
:03004300021A1B83
:03004B00021A1E78
:03005300021A216D
:03005B00021A2462
:03006300021A2757
:03006B00021A2A4C
:03007300021A2D41
:10060000E4F5D9E5EF7480F5FF7402F5EF787FE447
:10061000F6D8FD9000007F007E04E4F0A3DFFCDE4E
:07062000FA75817802066201
:1006270002129BE493A3F8E493A34003F68001F23C
:1006370008DFF48029E493A3F85407240CC8C333D4
:10064700C4540F4420C8834004F456800146F6DFA3
:10065700E4800B01020408102040809037FEE47EFE
:10066700019360BCA3FF543F30E509541FFEE49398
:10067700A360010ECF54C025E060A840B8E493A35F
:10068700FAE493A3F8E493A3C8C582C8CAC583CA8A
:10069700F0A3C8C582C8CAC583CADFE9DEE780BE42
:01381B0000AC
:100FE500E709F608DFFA8046E709F208DFFA803EEE
:100FF50088828C83E709F0A3DFFA8032E309F608DB
:10100500DFFA8078E309F208DFFA807088828C8342
:10101500E309F0A3DFFA806489828A83E0A3F608F6
:10102500DFFA805889828A83E0A3F208DFFA804CD0
:1010350080D280FA80C680D4806980F280338010A7
:1010450080A680EA809A80A880DA80E280CA803310
:1010550089828A83ECFAE493A3C8C582C8CCC58388
:10106500CCF0A3C8C582C8CCC583CCDFE9DEE78058
:101075000D89828A83E493A3F608DFF9ECFAA9F0D7
:10108500EDFB2289828A83ECFAE0A3C8C582C8CC2D
:10109500C583CCF0A3C8C582C8CCC583CCDFEADE46
:1010A500E880DB89828A83E493A3F208DFF980CCA8
:1010B50088F0EF60010E4E60C388F0ED2402B404A1
:1010C5000050B9F582EB2402B4040050AF23234548
:0610D50082239010357328
:1010DB00BB010689828A83E0225002E722BBFE0213
:0910EB00E32289828A83E4932246
:1010F400BB010989828A83F8E028F022500327F78C
:1011040022BBFE05F8E328F3228A838982F8E4935C
:0211140028228F
:10111600BB010689828A83F0225002F722BBFE01B8
:02112600F322B2
:10112800EF8DF0A4A8F0CF8CF0A428CE8DF0A42EDB
:02113800FE2295
:10113A00BC000BBE0029EF8DF084FFADF022E4CC99
:10114A00F875F008EF2FFFEE33FEEC33FCEE9DEC62
:10115A00984005FCEE9DFE0FD5F0E9E4CEFD22EDA8
:10116A00F8F5F0EE8420D21CFEADF075F008EF2FF2
:10117A00FFED33FD4007985006D5F0F222C398FDE3
:05118A000FD5F0EA2280
:10118F00C2D5EC30E709B2D5E4C39DFDE49CFCEE7B
:10119F0030E715B2D5E4C39FFFE49EFE12113AC3A8
:1011AF00E49DFDE49CFC800312113A30D507C3E4A3
:0611BF009FFFE49EFE22EA
:1011C500C5F0F8A3E028F0C5F0F8E58215827002B5
:0611D5001583E038F02252
:1011DB00A3F8E0C5F025F0F0E582158270021583C7
:0611EB00E0C838F0E82224
:0C11F100A42582F582E5F03583F5832209
:1011FD00FAE6FB0808E6F925F0F618E6CA3AF622F3
:09120D00E0FBA3E0FAA3E0F922E2
:10121600F8E0FBA3A3E0F925F0F0E5821582700261
:071226001583E0FA38F02205
:09122D00EBF0A3EAF0A3E9F022C2
:0C123600E493FB740193FA740293F92214
:10124200D083D082F8E4937012740193700DA3A33B
:1012520093F8740193F5828883E47374029368604F
:06126200EFA3A3A380DF4F
:061268008A838982E47311
:100C8000E51A241EF582E43401F583E0051A22906A
:100C9000011B30070390011EE475F00112121602C9
:100CA00010DB2000E97F2ED2008018EF540F249033
:100CB000D43440D4FF30040BEF24BFB41A005003E7
:100CC0002461FFE51B6002151B051EE51E70020571
:100CD0001D30070E90011BE475F001121216EF0291
:100CE00011160235BE7403D2078003E4C207F51A59
:100CF00090011B12122DE4F51BF51DF51EE51B607E
:100D0000077F20120CC380F5751CFFC201C200C210
:100D100002C203C205C206C208120C8FFF700D305A
:100D200007057F00120CD4AF1EAE1D22B4255FC292
:100D3000D5C204120C8FFF24D0B40A00501A75F0EB
:100D40000A781B30D50508B6FF0106C6A426F62092
:100D5000D5047002D20380D924CFB41A00EF500416
:100D6000C2E5D204020ED5D20180C6D20080C0D224
:100D70000280BCD2D580BAD20580B47F20120CC3C9
:100D80002002077401B51B0040F1120C80FF120C09
:100D9000C3020CFDD208D2068095120C80FB120C07
:100DA00080FA120C80F94A4B700679A67A0F7BFF05
:100DB00020022EE51B602A7E008E827583001212AF
:100DC0006E60060EEE651C70F0C2D5EBC0E0EAC0A6
:100DD000E0E9C0E0EE120F1CD0E0F9D0E0FAD0E07C
:100DE000FB1210DBFF60AAEBC0E0EAC0E0E9C0E064
:100DF000120CC3D0E02401F9D0E03400FAD0E0FBBB
:100E0000E51C0460DCD51CD980877BFF7A0F79183C
:100E1000D202809C791080027908C206C20880083C
:100E2000D2D5790A8004790AC2D5E51C047002F58E
:100E30001CE4FAFDFEFF120C80FC7B08200113125B
:100E40000C80FD7B1030000A120C80FE120C80FF1B
:100E50007B20EC3382D592D55013C3E43000069F3B
:100E6000FFE49EFEE42001039DFDE49CFCE4CBF83E
:100E7000C201EC700CCFCECDCCE824F8F870F38032
:100E800017C3EF33FFEE33FEED33FDEC33FCEB33F2
:100E9000FB994002FB0FD8E9EB300105F8D0E0C424
:100EA00048B201C0E00AEC4D4E4F78207B0070C282
:100EB000EAB51C0040BCC0E0120F1ED0F0D0E0200C
:100EC0000104C4C0E0C4B201C0F0120CACD0F0D533
:100ED000F0EB020CFD1212420D9A530E14580D6BDA
:100EE0004C0D67420E184F0E20440E20490D8043D2
:080EF0000E26550E0A460E0AFB
:100EF800450E0A470FC6500D6F2D0D732E0D962BFC
:100F08000D77230D94200FAF2A0D2F4800000D8E6A
:100F18003F3F3F00790AA2D5200314300509B910D4
:100F2800020404B9080104A2D520060250010420D5
:100F380002689202B51B005034C0E07F20300319CC
:100F48007F30A20272067205500F120F75C202C2DC
:100F580006C205C2087F30800F300503E9C0E012E1
:100F68000CC3300503D0E0F9D0E0B51BCC30051731
:100F78007F30B9100C120CC37F583004077F78807B
:100F880003B90803120CC33002057F2D020CC37F7E
:100F9800202008F87F2B2006F322920280CF286EAB
:100FA800756C6C2900D201120C803001F8C20178EE
:100FB8001B30D50108F6020D2F2D50434958120C4D
:100FC800802403B405004001E4900FC193120CB4CF
:0D0FD800743A120CB4D203751B04020E14FF
:10126E00BB010CE58229F582E5833AF583E0225035
:10127E0006E92582F8E622BBFE06E92582F8E2227F
:0D128E00E58229F582E5833AF583E4932299
:1035BE00EFB40A07740D1235C9740A309811A89920
:1035CE00B8130CC2983098FDA899C298B811F6306D
:0735DE0099FDC299F5992245
:00000001FF
